:030000000219FDE5
:03000B000200A848
:03002B0002015D72
:03005B000202DCC2
:030073000202C2C4
:1000800002030406080C10182030406080040608A3
:100090000C10182030406080A0C000070F1F3F05E3
:1000A000050D050205030302C2AFC0D0C0E0206207
:1000B00017E5256002E473E525F4F58A758B00D217
:1000C00062D0E0D0D0D2AF3285268AC262E526F473
:1000D000602F758B00D0E0D0D0C293C297C295D26A
:1000E000AF32C293C297C295206E0C206609740E7F
:1000F000D5E0FDE57E4290758B00D0E0D0D0D2AF48
:1001000032758A00C28DD26201F701B730680520CE
:100110006602D29301B7306805206602D29701B714
:10012000306805206602D29501B7C29230680A2075
:100130006607740CD5E0FDD29301B7C29630680A09
:10014000206607740CD5E0FDD29701B7C2943068E1
:100150000A206607740CD5E0FDD29501B7C2AFC284
:10016000AD53E6EFC0D0C0E0D2D3D2AFC2CEE52AC5
:100170006007207449152A21BE7800790020742E6A
:10018000E580307E01F430E50278FF53DACF207E3F
:100190000343DA20307E0343DA10C2D8C271E5800F
:1001A000307E01F430E50279FFC3E89970CB30610D
:1001B00003752A18207403752A18885FD27020747A
:1001C0000DE52B6004152B21CE43DA01C2D8207037
:1001D000024130A85F206102C270207431C3E894EC
:1001E000F0400374F0F8E8C4540F28F87984B7039A
:1001F00002410EC313C3138721200802C313200A30
:1002000006C3C898F8410E28F8500374FFF8C3E8F5
:1002100095685003E568F88822E52D54066011E5DD
:1002200033C313C31324062522F52250037522FF7E
:10023000852224A824C3E52495644002A864882567
:10024000E56970024174C3E8AA699A5003E8FAE4C8
:10025000F9EAC333FBE56BF45B29400D256AF8E549
:100260006A6002156A400B41740AC3E56A9A50023B
:10027000056A78FF8826C3E52594404002D26420B1
:10028000CF0AD0E0D0D043E610D2AD32C2CF053A8B
:100290007801E52A6005307402152AC3E55F9401F0
:1002A000400575620041B8756300756C00E5622415
:1002B00001F56250037562FFD0E0D0D043E610D262
:1002C000AD32C2AFC0D053E67FC260759100855693
:1002D00094855795759104D0D0D2AF32C2AF53E612
:1002E000EFC2ADC0D0C0E0C0F0D2D3D2AFA8FBA95E
:1002F000FCC2D8307102614353DACF207E0343DA67
:1003000010307E0343DA20D271E580307E01F42084
:10031000E502611A88278928A16A53DACF207E0373
:1003200043DA20307E0343DA10C2D8C2713074023F
:10033000A1567800E580307E01F430E502A15688B0
:100340005FA13E53DACF207E0343DA20307E0343A1
:10035000DA10C271206102811C53DACF207E034380
:10036000DA10307E0343DA20C2D8D271885A895B12
:10037000C3E89558F8E99559F97B007E087A00C3DF
:10038000E8948CE994005005755E00810E88217810
:10039000A2E6A8216055C3E894C8E994005008E497
:1003A000D2E4FB7A0A61E9C3E89468E99401500851
:1003B000E4D2E3FB7A0F61E9C3E894D0E9940250F8
:1003C00008E4D2E2FB7A1E61E9C3E894A0E994054F
:1003D0005008E4D2E1FB7A3C61E9C3E89498E994DF
:1003E000085008E4D2E0FB7A787E00C3E8955CFC14
:1003F000E9955DFD30E70AECF42401FCEDF43400EE
:10040000FD755E00C3EC9AED9E5003755E01885C3D
:10041000895D855A58855B597802A13EC3E89527C6
:10042000F8E99528F9307C02A122307B02A1223024
:100430007A02A11B207502813FE9FDE8FC815EE99B
:10044000C313F9E813F8307902A11BE9C313F9E8E3
:1004500013F8307802A11BE9C313FDE813FC2061F7
:1004600026C3EC941CED940240028175ED7018C314
:0E047000EC94C850120529C3E529940A5002E5
:10047E00A156755F00D270A156E529600215297844
:10048E0088E6F97400207F087896B90302789EE614
:10049E0024FAFEE43400FFC3EC9EFCED9FFD9208AF
:1004AE00B90310A2085007207609D27681C13076A2
:1004BE0002C276A2085016B9030DECF42401FCED2D
:1004CE00F43400FD0204DB78007900A122B9031593
:1004DE00EC33FCED33FDC3EC940AFCED9400FD50BF
:1004EE00047C007D00C3EC94FFED9400400678FF81
:1004FE007900A122EC8575F0A4C5F0A2F733F87946
:10050E0000400302053E78FF790002053EE9C31361
:10051E00F9E813F8307C0EE9600278FFC3E813386F
:10052E00F8E43400F9C3E894FFE99400400278FF40
:10053E00885FD270206102A156741FF4552F4BF5BF
:10054E002FC274EB7002D274752A18307403752A98
:10055E000A306102A16A20740353DAFE2074037517
:10056E002B06D0F0D0E0D0D0D2AD43E610327901D8
:10057E0002059A790302059A790A02059A791E02F2
:10058E00059A796402059A79C802059A7817E4D516
:10059E00E0FDD8FAD9F6227A147B780205C17A10DA
:1005AE007B8C0205C17A0D7BB40205C17A0B7BC828
:1005BE000205C17902B27DE4C296D5E0FDD297D58F
:1005CE00E0FDC297D5E0FDD296D5E0FDD293E5765B
:1005DE00D5E0FDC2937496D5E0FDD9D9EAF8D5E001
:1005EE00FDD8FBDBCEC29622C37C007D0075F000E9
:1005FE0005F0EA33FAEB33FB50F6EB13FBEA13FA92
:10060E00C3E9FFE8FEE89AF8E99BF95004EFF9EE2A
:10061E00F8B3EC33FCED33FDD5F0DFEDF9ECF82259
:10062E00E889F08A20D2D4F8A9F07B0030F70B7B52
:10063E00FFF42401F8E9F43400F9E88520F0A4ADC4
:10064E00F0F8E98520F0A4AFF0FEED2EF974003F2E
:10065E00FA7C04C3EA13FAE913F9E813F8DCF48B15
:10066E00F030F70AE8F42401F8E9F43400F9E889E7
:10067E00F0C2D4F8A9F02222C3E54113F9E54013E4
:10068E00F8C3E54598F8E54699F9500CC3E894800F
:10069E00E994FF40160206BDC3E8947FE99400502A
:1006AE00030206BD787F79000206BD788079FF8847
:1006BE004A894B22E54A2547F8E54B3548F9854BE3
:1006CE0020E4300701F43549FA30E709C3EA94F023
:1006DE0040150206FBC3EA940F50030206FB78FF97
:1006EE0079FF7A0F0206FB780079007AF0C3E524D1
:1006FE009564500AC374019524500B020719E54BFB
:10070E0020E70E020719E54B30E706884789488A2D
:10071E00492278A4E6FAC3E54A33F8E54B33F9D11A
:10072E002EE930E70BC3E89480E994FF4013E153C0
:10073E00C3E8947FE994005002E153787F7900E199
:10074E0053788079FFE820E715C3E52398F8400930
:10075E00C3E89401400302077A780102077AE8F4AD
:10076E0024012523F8400302077A78FF884C22786B
:10077E00A5E6FAA848A949D12EE930E70CC3E894BA
:10078E0001E994FF40160207AEC3E894FFE9940016
:10079E0050030207AE78FF79000207AE780179FFA9
:1007AE00E920E715C3E54C98F84009C3E8940140E9
:1007BE00030207D578010207D5E8F42401254CF889
:1007CE0040030207D578FF88242278FFC26420698F
:1007DE003D206A12D264C3E541940A4009C3E5255F
:1007EE0094405002C26479A1E76023E541601F7412
:1007FE00FF8541F0848539F0306A0375F005A4F861
:10080E00C5F0600278FFC3E895675002A867886656
:10081E0022C3E5409440E5419401E566500314017E
:10082E0030046002F566220208382275E8902278BC
:10083E0083E6FFE5E820ECF7A8BDA9BE0573C3E586
:10084E007394084052757300E9FA79A0E76044EAA0
:10085E007007E574601B020873C3E895746010E5B9
:0F086E00745006600C1402087F0460F902087FC2
:10087D00E574F574C3946D401B7564C0C394044056
:10088D0013756480C39404400B756440C394044095
:10089D000375640075BB0822E564F460020564E528
:1008AD0073B4070375BB1022743279A687F0A4C503
:1008BD00F0A2F733F8C3E895644002A86488228853
:1008CD0024882588268867227540007541F022C24C
:1008DD00AF75C820A8CCA9CDAA3A30CF010A75C8EA
:1008ED0024D2AFAB3BAC3C883B893CC3E89BF8E9D9
:1008FD009C206908F930670221F1214EAD3D8A3DFA
:10090D00F9EA9DFA600478FF79FFAE3EAF3F8B3E6A
:10091D008C3FC3EC9FFCC3E99CF542A83BA93CC3AB
:10092D00E89EF8E99FF9C3E54113FBE54013FAE8AA
:10093D002AF540E93BF54150067540FF7541FF2111
:10094D0098AA40AB41AC40AD417E047F02C3EB940D
:10095D000440021E1FC3EB940840021E1FC3ED137B
:10096D00FDEC13FCDEF7C3EA9CFAEB9DFBEF60098F
:10097D00C3E913F9E813F8DFF7EA28FAEB39FB8A34
:10098D00408B4150067BFF8B408B41C3EB94025053
:10099D0002D2673069047F0321C37892E6FFC3E575
:1009AD0037948240110FC3E53794A040010FC3EF78
:1009BD00940640027F057E06E541C4540FF9E541DA
:1009CD00C454F0F8E540C4540F28F8C3E89EFAE982
:1009DD009400FB4009C3EA9402EB940050047A02A0
:1009ED00E4FB413DAA40AB41EBC4FEEAC4540F4EBB
:1009FD00FCC3EA9CFAEB9400FBC3E813C313F8EABB
:100A0D0028FAEB3400FB8A408B41C3EB9402400281
:100A1D00C2677806EBC4FE7B00EAC4540F4EFAC3DE
:100A2D00EA98FA4005C3940250027A027892E6FFE2
:100A3D00306002413D855256855357D26043E68062
:100A4D00C3E49AF8E49BF930670241D7E8FAE9FB71
:100A5D00D3E913FDE813FC88528953C3EF94036067
:100A6D0038EF20E00DE82CF8E93DF9ECFAEDFB024A
:100A7D000A92E828F8E939F9C3E82402F8E93400C4
:100A8D00F97AFE7BFFC3EF9403400E8A548B558891
:100A9D004E894F8C508D51610B885489558A4E8BE0
:100AAD004F8C508D51306920C3E53394034019E5C7
:100ABD0042A2E713F8E555F4240138400B20E7086E
:100ACD007554FFF42401F555610BE8FAD3E813FCD6
:100ADD008852C3EF94036020EF20E007E82CF8EC78
:100AED00FA41F7E8282402F87AFEC3EF9403400890
:100AFD008A54884E8C50610B88548A4E8C50E56B0D
:100B0D00C3335002646BF56B3060026115753402AE
:100B1D00D26043E680E52D54066026A840A941C366
:100B2D00E913F9E813F8C2AF53E67F759100C3E4FA
:100B3D0098F594E499F595759104D26043E680D2C9
:100B4D00AF22D265754400752000306B03752040CF
:100B5D00020B6ED265754400752040306B03752015
:100B6D0000D2AF7801206722E52D54066002C265E0
:100B7D00C3E5419405401378029405400878039429
:100B8D000540027806306902780A206019E5446054
:100B9D001530690AC3E53394034003D53406D2AF4B
:100BAD00D26C813F711DD2AF0000C2AF206726E528
:100BBD0041C3FB940F40027B0FEB240530730123DF
:100BCD00306A02742820620123F93069027982E5C6
:100BDD008BC39940B50544E59B5440B5200281294E
:100BED0030690A08C3E8940A40010861972065023C
:100BFD00616EC26553E67F75910030671075940084
:100C0D007595FE759104D26043E680616EAE40AF7E
:100C1D0041C3E49EF594E49FF5958110C3E53394AB
:100C2D00025002616E306502616ED802813D61979E
:100C3D00C26C53E67F7591008554948555957591D9
:100C4D0004854E56854F57D26043E680D2AFE52DD1
:100C5D0054066008206A020533020C79306C0D20B1
:0F0C6D006B0A206507158115810214F0227800AB
:100C7C003064053065027801E53775F007A4F9E5B5
:100C8C00F028F5F0E9A2F013A2F113A2F213F53754
:100C9C00C394785003753778C3E53795384008D23C
:100CAC0066C293C297C29530600281B38550568557
:100CBC005157D26043E68022207D11C2AF754302AA
:100CCC00C296D292D2AF759F11020E93C2AF7543EA
:100CDC0002C296D294D2AF759F11020E933072431A
:100CEC00207D20C2AF75430390013B757E40C295B9
:100CFC00C294306204D297A107D296D2AF759F10DE
:100D0C00020E93C2AF75430390013B757E40C293B4
:100D1C00C292306204D297A127D296D2AF759F139C
:100D2C00020E93207D17C2AF754303900116C29536
:100D3C00306202D297D2AF759F10020E93C2AF757C
:100D4C004303900116C293306202D297D2AF759FC3
:100D5C0013020E93207D11C2AF754304C292D2943C
:100D6C00D2AF759F13020E93C2AF754304C294D2D7
:100D7C0092D2AF759F10020E93307243207D20C229
:100D8C00AF75430590012A757E04C297C2963062F6
:100D9C0004D293A1A3D292D2AF759F11020E93C22B
:100DAC00AF75430590014C757E10C297C2963062A8
:100DBC0004D295A1C3D294D2AF759F11020E932089
:100DCC007D17C2AF75430590010CC297306202D2F9
:100DDC0093D2AF759F11020E93C2AF75430590016C
:100DEC0020C2973062EBD295D2AF759F11020E9351
:100DFC00207D11C2AF754306C294D296D2AF759FB7
:100E0C0010020E93C2AF754306C292D296D2AF7542
:100E1C009F13020E93307242207D20C2AF754301A6
:100E2C0090014C757E10C293C292306204D295C16F
:100E3C003FD294D2AF759F13020E93C2AF7543018C
:100E4C0090012A757E04C295C294306204D293C17B
:100E5C005FD292D2AF759F10C193207D16C2AF7531
:100E6C004301900120C293306202D295D2AF759F9C
:100E7C0013C193C2AF75430190010CC2953062024D
:100E8C00D293D2AF759F10C2662290010A757E0074
:100E9C00C293C297C295C292C296C294C262227881
:100EAC008076FF0876FF0876FF0876FF0876030841
:100EBC007604087608087601087601087601788CA5
:100ECC0076010876FF0876FF0876FF0876FF08762D
:100EDC00FF0876030876FF0876FF0876FF0876256C
:100EEC000876D00876FA0876FA0876040876FF08B1
:100EFC00760108760008767A0876FF08760108767F
:100F0C0001087600087603227887E6FFC27278889B
:100F1C00E6C394036008C27DE630E102D27DC27E56
:100F2C007889E630E102D27EC3EF94026008758EB8
:100F3C0001D273020F47758E00C273227880E614BB
:100F4C009000809378A4F67881E6149000809378D2
:100F5C00A5F67886E61490008D9378A6F6789CE634
:100F6C007538FF75390CB402067538A075390AB49A
:100F7C00030675388275390578A3E61490009A93A8
:100F8C00F569D19622227896E6FA7897E6FB78886E
:100F9C00E6B40305C3EB940EFB307F047A007BFFB1
:100FAC00C3EB9AFCC3948250027C82757500057564
:100FBC00EC8575F0A4C3E5F0947D40F222D27FF16C
:100FCC009212058B7A007B007C10120581E55F2A5A
:100FDC00FA74003BFBDCF37C04C3EB13FBEA13FA5F
:100FEC00DCF7FEC27FF19222E5EF20E603752000CC
:100FFC000520903FFFE520146006901DFF14600053
:10100C009304600375EF1253D9BF7581C043FF8001
:10101C0012057C75EF0243B203E5B3240420E70DFF
:10102C00F521E5E320E0068521B343E301120E969A
:10103C007580FF75A40075F1B275D4DF75900375DA
:10104C00A5FC75F2FC75D50375A60175E241E4F8B3
:10105C00F6D8FD756B01120EAB12153278988676A8
:0E106C00753001C2AF1205951205A512058B55
:10107A001205AC12058B1205B312058B12164B1210
:10108A000595120595120590C2AF78FA79FA30855E
:10109A0007D9FBD8F7021C00120F14120F48120FBF
:1010AA0091120F9278988676120E967588507589E5
:1010BA001275C82475910475D84075A82275B802AE
:1010CA0075E690759B80759D0075D10E75BC587537
:1010DA00BB0875BA1175E88012057CD2AF120835C3
:1010EA0053DACF207E0343DA20307E0343DA1043FB
:1010FA00DA01C2D8C271120595D2617B037A0CE576
:10110A005E70077A0CDB0302109212058B207003C3
:10111A00021092C270E55FC3940240E1E52F541FAA
:10112A00856160F561B560D5DAD5C26153DACF2041
:10113A007E0343DA20307E0343DA10C2D8C27178C4
:10114A00A2E67008D274E52F54E0F52FC27575290E
:10115A0000120590307409C3E529940A4002D27539
:10116A0012058178023074027800C3E55F9840F076
:10117A00C2AF1205A51205A51205A5D2AF12059593
:10118A00754D007888E6B403024172120581788CA5
:10119A00E6C394015003021272E530C3940150036E
:1011AA00021272207435C3E55F94FF500302127273
:1011BA00C2AF1205BAD2AF120590C3E55F940150CF
:1011CA00EFC2AF1205A51205861205A5D2AF120508
:1011DA0090C3E55F94FF40E90216D07F05D27F12E3
:1011EA000F92120590C2AFC27F120F92AE5FC3E593
:1011FA005F947FD2AF407B12057CC2AF1205BAD290
:10120A00AFDFDA120FC9C3EE94057897F612059587
:10121A001215741216537F0AD27F120F921205907A
:10122A00C2AFC27F120F92AE5FC3E55F947FD2AFA7
:10123A0050E412057CC2AF1205A51205861205A557
:10124A00D2AFDFD4120FC9EE24057896F6120595AF
:10125A00121574121682120590120F92C3E55F944A
:10126A00FF500221AD0216D0C3E55F954D400385BC
:10127A005F4D12059078017988E7B403027805C3B7
:10128A00E55F984002218DC2AF1205BA1205BA1263
:10129A0005BAD2AF120595753000E4F531F532057D
:1012AA0031E531F470390532789AE678191460120A
:1012BA00783214600D787D14600878FA146003752A
:1012CA003200C3E53298401715327531B4789986E1
:1012DA0076C2AF1205BAD2AF789886761205901206
:1012EA000586E52A7005307402019278012074029D
:1012FA007806C3E55F9840A77888E6C3940360033D
:10130A00120590E52A7003021092C2AF120E96E4FB
:10131A00F522F523F524F525F526F56AD2AF788569
:10132A00E6C333F568E4F545F546F547F548F5496A
:10133A00F573F52CF52DF53775730875BB10120585
:10134A007C120839E5E820ECFBA8BDA9BEE97001CA
:10135A00F8887412083D75730875BB107887E6FE25
:10136A007602120F147887EEF6C2AF7564FF120880
:10137A00B5852264852265852266D2AF75220175FC
:10138A00240175250175260185636C756D017888C0
:10139A00E6B40307C27D307602D27DD268D269757F
:1013AA003300120DFC120E211208D51208DC1208A5
:1013BA00D51208DC1208D50213D1C2AF120F14D20B
:1013CA00AF75730075BB08120B60120685120C7A92
:1013DA00120CC41208DC120B4F306D031206862061
:1013EA0067031207D830670312081F120C7A120C0F
:1013FA00E91208DC120B60306D031206C2120C7A75
:10140A00120D601208DC120B4F306D031207201206
:10141A000C7A120D851208DC120B60306D0312076C
:10142A007D120C7A120DFC1208DC120839120B4FCD
:10143A00120C7A120E2112083D1208DC3069322091
:10144A006B2F85676485676585636C756D0179188F
:10145A007A0CC3E53399400CC269D26A8A3575643D
:0E146A00FF02147BC3E55F940140030213D11F
:101478000214F8306A1B206B18E535147004C26A30
:1014880061C4F535C3E55F940140030213D102142A
:10149800F8753600C3E5627882985054307404E5D4
:1014A8002A604D7888E6B40317207D0520760781E9
:1014B800C830760281C8206B07D26B8567648110BB
:1014C80078F0306B058567647820C3E54198500251
:1014D80061D1306B1BC26BC27D307602D27DD26A7D
:1014E80075351285676461D10536E55F600281FB59
:1014F800753600C2AF120E967887E6FE7602120F96
:10150800147887EEF6E4F522F523F524F525F5267B
:10151800F568C268D2AF12057C120E96307409C302
:10152800E53694054002019241A4901A0D782012E4
:1015380015B6E520B45A0CA31215B6E520B4A503D8
:10154800021554120EAB121574021573901A037813
:10155800807B0A1215B6A308DBF9901A0F788C7BEA
:10156800181215B6A308DBF9901A2722C2AF121574
:10157800F51215CF901A00740E1215BBA37404123D
:1015880015BBA374141215BB901A0378807B0A123A
:1015980015BAA308DBF9901A0F788C7B181215BAC4
:1015A800A308DBF91216081215E6901A2722E4930D
:1015B800F622E6438F01538FFD75EF0275B7A575C7
:1015C800B7F1F0538FFE22438F02438F0175EF026C
:1015D80075B7A575B7F1901A0DF0538FFC22901AC4
:1015E8000D745AB1BB901A0E74A5B1BB227A30792A
:1015F800D07820901A40B1B6E520F709A3DAF7228F
:101608007A3079D0901A40E7B1BB09A3DAF922AB56
:1016180077A878BB01027984BB02027985BB0302F3
:101628007986BB04027992BB05027987BB060279E9
:10163800A3BB0702799CBB08027988BB0902798998
:10164800E8F7227C05120595DCFB22C2AF1205A53E
:101658001205AC1205B31205BA1205861205A512B9
:1016680005AC1205B31205BA1205861205A51205B6
:10167800AC1205B31205BAD2AF22C2AF1205BA1224
:1016880005B31205AC1205A51205861205BA120596
:10169800B31205AC1205A51205861205BA1205B3D8
:1016A8001205AC1205A5D2AF22AE77AF78C2AF1241
:1016B80005A51205A51205A5120586DEF21205BAC2
:1016C800120586DFF8D2AF22D153D14BD14B7577B3
:1016D80001757801757900D1B17C05AD5F1205956A
:1016E800C3ED955F70F5C3E55F9401400AC3E55FFC
:1016F80094FF403202170CD117B174D153C2AF75A1
:10170800EF12D14BDCD50579C3E5799403500280FB
:10171800C6D14B0578E5771490009F93F808C3E588
:101728007898500280AED14BD14B0577C3E57794BA
:101738000A5002809C120EABB174C2AF75EF12D181
:011748004B55
:0319FD00020FF4E2
:101A00000E0414FFFFFFFF0304080101015AA501A2
:101A1000FFFFFFFFFF03FFFFFF25D0FAFA04FF01DE
:081A2000007AFF01010003FF41
:101A4000235475726E696779363041232020202037
:101A500023424C48454C4923463333302320202031
:101A60002020202020202020202020202020202076
:101C0000C2AFC2D353D9BF7581C043B20343FF8073
:101C1000752438752503B1C975EF0275E24043F1AB
:101C20002053A4DF75D400D2857DFA780379E67C51
:101C300010752200752300901DD67B0675249875BB
:101C400025013085028142208508D8FBD9F9DCF7CF
:101C500081B4308508D8FBD9F9DCF781B4B189E4C7
:101C600093A3C39A6004DDC381B4DBDBB17B600264
:101C7000812B7B08E493FAA3B15CDBF87A30B15C8A
:101C8000752200752300B17BEAFCEBFDC3ED94FEE9
:101C9000400EB17B8A278B28ED30E0048A828B834B
:101CA000B17B7AC270D8C3ED94FE601350CEBD00F4
:101CB00025EC60097520007521FF0200008100A855
:101CC00027A9280809D804D90281D3B17FEA89AAB3
:101CD000F281C50D81A0C3ED94035049EDA2E092BD
:101CE000007AC5C3E5829400E583941C50902000DF
:101CF00010438F02438F0175B7A575B7F1F030001F
:101D00001FA827A9280809438F01538FFDD804D99C
:101D100002A12089AAE275B7A575B7F1F0A3A10DBC
:101D2000538FFC817C7AC1BD030CE493A3FAB140CC
:101D3000DCF8B138817C817EAA22AB23B15CEBFA5E
:101D4000EA6222752608C3E52313F523E52213F57D
:101D50002250066323A0632201D526EAB1C9B1C986
:101D600075260AEAF4200102D285300102C285B14B
:101D7000C9C3134002C201D526EB22B17FEAFB2082
:101D80008502A17F308502A184752608AE24AF2587
:101D9000C3EF13FFEE13FEB1CDB1C9C3EA13308513
:101DA000024480FA30E703632201C3E52313F523DD
:101DB000E52213F52250066323A0632201D526D91C
:101DC000E52265236523F52222AE24AF250E0FDE22
:101DD000FEDFFCD20122424C48656C693437316326
:041DE000F3300601D5
:00000001FF
